
 OLE2

 Start     Length     Name                   Class
 0001:0000 00000H     O_Init                 CODE
 0001:0000 052F6H     SEG_CODE_TEXT          CODE
 0002:0000 00B3CH     _TEXT                  CODE
 0003:0000 00160H     COMDAT_SEG1            CODE
 0004:0000 00010H     NULL                   BEGDATA
 0004:0010 0030EH     _DATA                  DATA
 0004:031E 0000EH     CDATA                  DATA
 0004:032C 00000H     XIFB                   DATA
 0004:032C 00000H     XIF                    DATA
 0004:032C 00000H     XIFE                   DATA
 0004:032C 00000H     XIB                    DATA
 0004:032C 00000H     XI                     DATA
 0004:032C 00000H     XIE                    DATA
 0004:032C 00000H     XPB                    DATA
 0004:032C 00000H     XP                     DATA
 0004:032C 00000H     XPE                    DATA
 0004:032C 00000H     XCB                    DATA
 0004:032C 00000H     XC                     DATA
 0004:032C 00000H     XCE                    DATA
 0004:032C 00000H     XCFB                   DATA
 0004:032C 00000H     XCFCRT                 DATA
 0004:032C 00000H     XCF                    DATA
 0004:032C 00000H     XCFE                   DATA
 0004:032C 00000H     XIFCB                  DATA
 0004:032C 00000H     XIFU                   DATA
 0004:032C 00000H     XIFL                   DATA
 0004:032C 00000H     XIFM                   DATA
 0004:032C 00000H     XIFCE                  DATA
 0004:032C 00000H     DBDATA                 DATA
 0004:032C 00000H     CONST                  CONST
 0004:032C 00008H     HDR                    MSG
 0004:0334 0016EH     MSG                    MSG
 0004:04A2 00002H     PAD                    MSG
 0004:04A4 00001H     EPAD                   MSG
 0004:04A6 0003CH     _BSS                   BSS
 0004:04E2 00000H     XOB                    BSS
 0004:04E2 00000H     XO                     BSS
 0004:04E2 00000H     XOE                    BSS
 0004:04E2 00000H     XOFB                   BSS
 0004:04E2 00000H     XOF                    BSS
 0004:04E2 00000H     XOFE                   BSS

 Origin   Group
 0004:0   DGROUP

 Address   Export                  Alias

 0001:3000 ?AddRef@CMemBytes@@VEAKXZ  ?AddRef@CMemBytes@@VEAKXZ
 0001:23A2 ?AddRef@CMemStm@@VEAKXZ  ?AddRef@CMemStm@@VEAKXZ
 0001:3B88 ?AddRef@CMMB@@VEAKXZ    ?AddRef@CMMB@@VEAKXZ
 0001:35F2 ?AddRef@CMMS@@VEAKXZ    ?AddRef@CMMS@@VEAKXZ
 0001:2B48 ?Clone@CMemStm@@VEAPEXPEPEUIStream@@@Z  ?Clone@CMemStm@@VEAPEXPEPEUIStream@@@Z
 0001:2A3A ?Commit@CMemStm@@VEAPEXK@Z  ?Commit@CMemStm@@VEAPEXK@Z
 0001:28AA ?CopyTo@CMemStm@@VEAPEXPEUIStream@@U_ULARGE_INTEGER@@PEU3@2@Z  ?CopyTo@CMemStm@@VEAPEXPEUIStream@@U_ULARGE_INTEGER@@PEU3@2@Z
 0001:3458 ?Create@CMemBytes@@TAPEV1@I@Z  ?Create@CMemBytes@@TAPEV1@I@Z
 0001:2BAE ?Create@CMemStm@@TAPEV1@I@Z  ?Create@CMemStm@@TAPEV1@I@Z
 0001:3F58 ?Create@CMMB@@TAPEV1@PEVCMemBytes@@@Z  ?Create@CMMB@@TAPEV1@PEVCMemBytes@@@Z
 0001:39CA ?Create@CMMS@@TAPEV1@PEVCMemStm@@@Z  ?Create@CMMS@@TAPEV1@PEVCMemStm@@@Z
 0001:3F48 ?DisconnectObject@CMMB@@VEAPEXK@Z  ?DisconnectObject@CMMB@@VEAPEXK@Z
 0001:39BA ?DisconnectObject@CMMS@@VEAPEXK@Z  ?DisconnectObject@CMMS@@VEAPEXK@Z
 0001:32E2 ?Flush@CMemBytes@@VEAPEXXZ  ?Flush@CMemBytes@@VEAPEXXZ
 0001:3C7C ?GetMarshalSizeMax@CMMB@@VEAPEXAFUGUID@@PEXK1KPEK@Z  ?GetMarshalSizeMax@CMMB@@VEAPEXAFUGUID@@PEXK1KPEK@Z
 0001:36E8 ?GetMarshalSizeMax@CMMS@@VEAPEXAFUGUID@@PEXK1KPEK@Z  ?GetMarshalSizeMax@CMMS@@VEAPEXAFUGUID@@PEXK1KPEK@Z
 0001:3C2C ?GetUnmarshalClass@CMMB@@VEAPEXAFUGUID@@PEXK1KPEU2@@Z  ?GetUnmarshalClass@CMMB@@VEAPEXAFUGUID@@PEXK1KPEU2@@Z
 0001:3696 ?GetUnmarshalClass@CMMS@@VEAPEXAFUGUID@@PEXK1KPEU2@@Z  ?GetUnmarshalClass@CMMS@@VEAPEXAFUGUID@@PEXK1KPEU2@@Z
 0001:336E ?LockRegion@CMemBytes@@VEAPEXU_ULARGE_INTEGER@@0K@Z  ?LockRegion@CMemBytes@@VEAPEXU_ULARGE_INTEGER@@0K@Z
 0001:2A5A ?LockRegion@CMemStm@@VEAPEXU_ULARGE_INTEGER@@0K@Z  ?LockRegion@CMemStm@@VEAPEXU_ULARGE_INTEGER@@0K@Z
 0001:3CD0 ?MarshalInterface@CMMB@@VEAPEXPEUIStream@@AFUGUID@@PEXK2K@Z  ?MarshalInterface@CMMB@@VEAPEXPEUIStream@@AFUGUID@@PEXK2K@Z
 0001:374E ?MarshalInterface@CMMS@@VEAPEXPEUIStream@@AFUGUID@@PEXK2K@Z  ?MarshalInterface@CMMS@@VEAPEXPEUIStream@@AFUGUID@@PEXK2K@Z
 0001:2F3A ?QueryInterface@CMemBytes@@VEAPEXAFUGUID@@PEPEX@Z  ?QueryInterface@CMemBytes@@VEAPEXAFUGUID@@PEPEX@Z
 0001:22DC ?QueryInterface@CMemStm@@VEAPEXAFUGUID@@PEPEX@Z  ?QueryInterface@CMemStm@@VEAPEXAFUGUID@@PEPEX@Z
 0001:3AD0 ?QueryInterface@CMMB@@VEAPEXAFUGUID@@PEPEX@Z  ?QueryInterface@CMMB@@VEAPEXAFUGUID@@PEPEX@Z
 0001:3538 ?QueryInterface@CMMS@@VEAPEXAFUGUID@@PEPEX@Z  ?QueryInterface@CMMS@@VEAPEXAFUGUID@@PEPEX@Z
 0001:2434 ?Read@CMemStm@@VEAPEXPIXKPEK@Z  ?Read@CMemStm@@VEAPEXPIXKPEK@Z
 0001:3092 ?ReadAt@CMemBytes@@VEAPEXU_ULARGE_INTEGER@@PIXKPEK@Z  ?ReadAt@CMemBytes@@VEAPEXU_ULARGE_INTEGER@@PIXKPEK@Z
 0001:3022 ?Release@CMemBytes@@VEAKXZ  ?Release@CMemBytes@@VEAKXZ
 0001:23C4 ?Release@CMemStm@@VEAKXZ  ?Release@CMemStm@@VEAKXZ
 0001:3BAA ?Release@CMMB@@VEAKXZ   ?Release@CMMB@@VEAKXZ
 0001:3614 ?Release@CMMS@@VEAKXZ   ?Release@CMMS@@VEAKXZ
 0001:3EEC ?ReleaseMarshalData@CMMB@@VEAPEXPEUIStream@@@Z  ?ReleaseMarshalData@CMMB@@VEAPEXPEUIStream@@@Z
 0001:395E ?ReleaseMarshalData@CMMS@@VEAPEXPEUIStream@@@Z  ?ReleaseMarshalData@CMMS@@VEAPEXPEUIStream@@@Z
 0001:2A4A ?Revert@CMemStm@@VEAPEXXZ  ?Revert@CMemStm@@VEAPEXXZ
 0001:26D8 ?Seek@CMemStm@@VEAPEXU_LARGE_INTEGER@@KPEU_ULARGE_INTEGER@@@Z  ?Seek@CMemStm@@VEAPEXU_LARGE_INTEGER@@KPEU_ULARGE_INTEGER@@@Z
 0001:32F2 ?SetSize@CMemBytes@@VEAPEXU_ULARGE_INTEGER@@@Z  ?SetSize@CMemBytes@@VEAPEXU_ULARGE_INTEGER@@@Z
 0001:2822 ?SetSize@CMemStm@@VEAPEXU_ULARGE_INTEGER@@@Z  ?SetSize@CMemStm@@VEAPEXU_ULARGE_INTEGER@@@Z
 0001:338E ?Stat@CMemBytes@@VEAPEXPEUtagSTATSTG@@K@Z  ?Stat@CMemBytes@@VEAPEXPEUtagSTATSTG@@K@Z
 0001:2A7E ?Stat@CMemStm@@VEAPEXPEUtagSTATSTG@@K@Z  ?Stat@CMemStm@@VEAPEXPEUtagSTATSTG@@K@Z
 0001:337E ?UnlockRegion@CMemBytes@@VEAPEXU_ULARGE_INTEGER@@0K@Z  ?UnlockRegion@CMemBytes@@VEAPEXU_ULARGE_INTEGER@@0K@Z
 0001:2A6C ?UnlockRegion@CMemStm@@VEAPEXU_ULARGE_INTEGER@@0K@Z  ?UnlockRegion@CMemStm@@VEAPEXU_ULARGE_INTEGER@@0K@Z
 0001:3DC8 ?UnmarshalInterface@CMMB@@VEAPEXPEUIStream@@AFUGUID@@PEPEX@Z  ?UnmarshalInterface@CMMB@@VEAPEXPEUIStream@@AFUGUID@@PEPEX@Z
 0001:383A ?UnmarshalInterface@CMMS@@VEAPEXPEUIStream@@AFUGUID@@PEPEX@Z  ?UnmarshalInterface@CMMS@@VEAPEXPEUIStream@@AFUGUID@@PEPEX@Z
 0001:257C ?Write@CMemStm@@VEAPEXPJXKPEK@Z  ?Write@CMemStm@@VEAPEXPJXKPEK@Z
 0001:31CC ?WriteAt@CMemBytes@@VEAPEXU_ULARGE_INTEGER@@PJXKPEK@Z  ?WriteAt@CMemBytes@@VEAPEXU_ULARGE_INTEGER@@PJXKPEK@Z
 0001:080C BINDMONIKER             BINDMONIKER
 0001:2D06 CLONEMEMSTM             CLONEMEMSTM
 0001:4046 CMEMBYTESUNMARSHAL      CMEMBYTESUNMARSHAL
 0001:3AB8 CMEMSTMUNMARSHAL        CMEMSTMUNMARSHAL
 0001:09BE CREATEANTIMONIKER       CREATEANTIMONIKER
 0001:08A4 CREATEBINDCTX           CREATEBINDCTX
 0001:0774 CREATEDATAADVISEHOLDER  CREATEDATAADVISEHOLDER
 0001:079A CREATEDATACACHE         CREATEDATACACHE
 0001:0916 CREATEFILEMONIKER       CREATEFILEMONIKER
 0001:08CA CREATEGENERICCOMPOSITE  CREATEGENERICCOMPOSITE
 0001:212A CREATEILOCKBYTESONHGLOBAL  CREATEILOCKBYTESONHGLOBAL
 0001:0998 CREATEITEMMONIKER       CREATEITEMMONIKER
 0001:2C84 CREATEMEMSTM            CREATEMEMSTM
 0001:053A CREATEOLEADVISEHOLDER   CREATEOLEADVISEHOLDER
 0001:09E4 CREATEPOINTERMONIKER    CREATEPOINTERMONIKER
 0001:2D8E CREATESTREAMONHGLOBAL   CREATESTREAMONHGLOBAL
 0001:1E0C DBGDUMPCLASSNAME        DBGDUMPCLASSNAME
 0001:1DEC DBGDUMPEXTERNALOBJECT   DBGDUMPEXTERNALOBJECT
 0001:1DDE DBGDUMPOBJECT           DBGDUMPOBJECT
 0001:1DFA DBGISOBJECTVALID        DBGISOBJECTVALID
 0001:1D74 DBGLOGCLOSE             DBGLOGCLOSE
 0001:1D62 DBGLOGOPEN              DBGLOGOPEN
 0001:1DAC DBGLOGOUTPUTDEBUGSTRING  DBGLOGOUTPUTDEBUGSTRING
 0001:1D90 DBGLOGTIMESTAMP         DBGLOGTIMESTAMP
 0001:1D82 DBGLOGWRITE             DBGLOGWRITE
 0001:1D9E DBGLOGWRITEBANNER       DBGLOGWRITEBANNER
 0001:004C DLLGETCLASSOBJECT       DLLGETCLASSOBJECT
 0001:0390 DODRAGDROP              DODRAGDROP
 0001:1E1A DUMPALLOBJECTS          DUMPALLOBJECTS
 0001:08F0 GETCLASSFILE            GETCLASSFILE
 0001:0728 GETCONVERTSTG           GETCONVERTSTG
 0001:170A GETDOCUMENTBITSTG       GETDOCUMENTBITSTG
 0001:2240 GETHGLOBALFROMILOCKBYTES  GETHGLOBALFROMILOCKBYTES
 0001:2EA4 GETHGLOBALFROMSTREAM    GETHGLOBALFROMSTREAM
 0001:0A0A GETRUNNINGOBJECTTABLE   GETRUNNINGOBJECTTABLE
 0001:1F16 ISACCELERATOR           ISACCELERATOR
 0001:1DCC MAKEDEBUGSTREAM         MAKEDEBUGSTREAM
 0001:0832 MKPARSEDISPLAYNAME      MKPARSEDISPLAYNAME
 0001:087E MONIKERCOMMONPREFIXWITH  MONIKERCOMMONPREFIXWITH
 0001:0858 MONIKERRELATIVEPATHTO   MONIKERRELATIVEPATHTO
 0001:10C2 OLEBUILDVERSION         OLEBUILDVERSION
 0001:0644 OLECONVERTISTORAGETOOLESTREAM  OLECONVERTISTORAGETOOLESTREAM
 0001:0690 OLECONVERTISTORAGETOOLESTREAMEX  OLECONVERTISTORAGETOOLESTREAMEX
 0001:066A OLECONVERTOLESTREAMTOISTORAGE  OLECONVERTOLESTREAMTOISTORAGE
 0001:06B6 OLECONVERTOLESTREAMTOISTORAGEEX  OLECONVERTOLESTREAMTOISTORAGEEX
 0001:0156 OLECREATE               OLECREATE
 0001:0560 OLECREATEDEFAULTHANDLER  OLECREATEDEFAULTHANDLER
 0001:0586 OLECREATEEMBEDDINGHELPER  OLECREATEEMBEDDINGHELPER
 0001:017C OLECREATEFROMDATA       OLECREATEFROMDATA
 0001:023A OLECREATEFROMFILE       OLECREATEFROMFILE
 0001:01EE OLECREATELINK           OLECREATELINK
 0001:01A2 OLECREATELINKFROMDATA   OLECREATELINKFROMDATA
 0001:0214 OLECREATELINKTOFILE     OLECREATELINKTOFILE
 0001:0000 OLECREATEMENUDESCRIPTOR  OLECREATEMENUDESCRIPTOR
 0001:01C8 OLECREATESTATICFROMDATA  OLECREATESTATICFROMDATA
 0001:0026 OLEDESTROYMENUDESCRIPTOR  OLEDESTROYMENUDESCRIPTOR
 0001:196C OLEDOAUTOCONVERT        OLEDOAUTOCONVERT
 0001:04A2 OLEDRAW                 OLEDRAW
 0001:1344 OLEDUPLICATEDATA        OLEDUPLICATEDATA
 0001:043C OLEFLUSHCLIPBOARD       OLEFLUSHCLIPBOARD
 0001:06DC OLEGETAUTOCONVERT       OLEGETAUTOCONVERT
 0001:1DBA OLEGETCLASSID           OLEGETCLASSID
 0001:0416 OLEGETCLIPBOARD         OLEGETCLIPBOARD
 0001:435E OLEGETICONOFCLASS       OLEGETICONOFCLASS
 0001:405E OLEGETICONOFFILE        OLEGETICONOFFILE
 0001:10A2 OLEGETMALLOC            OLEGETMALLOC
 0001:0EB2 OLEINITIALIZE           OLEINITIALIZE
 0001:0456 OLEISCURRENTCLIPBOARD   OLEISCURRENTCLIPBOARD
 0001:04EE OLEISRUNNING            OLEISRUNNING
 0001:0260 OLELOAD                 OLELOAD
 0001:02AC OLELOADFROMSTREAM       OLELOADFROMSTREAM
 0001:0514 OLELOCKRUNNING          OLELOCKRUNNING
 0001:4838 OLEMETAFILEPICTFROMICONANDLABEL  OLEMETAFILEPICTFROMICONANDLABEL
 0001:031E OLENOTEOBJECTVISIBLE    OLENOTEOBJECTVISIBLE
 0001:0130 OLEQUERYCREATEFROMDATA  OLEQUERYCREATEFROMDATA
 0001:010A OLEQUERYLINKFROMDATA    OLEQUERYLINKFROMDATA
 0001:05F8 OLEREGENUMFORMATETC     OLEREGENUMFORMATETC
 0001:061E OLEREGENUMVERBS         OLEREGENUMVERBS
 0001:05D2 OLEREGGETMISCSTATUS     OLEREGGETMISCSTATUS
 0001:05AC OLEREGGETUSERTYPE       OLEREGGETUSERTYPE
 0001:04C8 OLERUN                  OLERUN
 0001:0286 OLESAVE                 OLESAVE
 0001:02D2 OLESAVETOSTREAM         OLESAVETOSTREAM
 0001:0702 OLESETAUTOCONVERT       OLESETAUTOCONVERT
 0001:03B6 OLESETCLIPBOARD         OLESETCLIPBOARD
 0001:02F8 OLESETCONTAINEDOBJECT   OLESETCONTAINEDOBJECT
 0001:047C OLESETMENUDESCRIPTOR    OLESETMENUDESCRIPTOR
 0001:502C OLESTDGETAUXUSERTYPE    OLESTDGETAUXUSERTYPE
 0001:4EB8 OLESTDGETUSERTYPEOFCLASS  OLESTDGETUSERTYPEOFCLASS
 0001:4B1E OLESTDICONLABELTEXTOUT  OLESTDICONLABELTEXTOUT
 0001:1E38 OLETRANSLATEACCELERATOR  OLETRANSLATEACCELERATOR
 0001:0FFE OLEUNINITIALIZE         OLEUNINITIALIZE
 0001:1CE4 OPENORCREATESTREAM      OPENORCREATESTREAM
 0001:0072 READCLASSSTG            READCLASSSTG
 0001:1056 READCLASSSTM            READCLASSSTM
 0001:00E4 READFMTUSERTYPESTG      READFMTUSERTYPESTG
 0001:07C0 READOLESTG              READOLESTG
 0001:1B3A READSTRINGSTREAM        READSTRINGSTREAM
 0001:0344 REGISTERDRAGDROP        REGISTERDRAGDROP
 0001:2D1C RELEASEMEMSTM           RELEASEMEMSTM
 0001:1784 RELEASESTGMEDIUM        RELEASESTGMEDIUM
 0001:036A REVOKEDRAGDROP          REVOKEDRAGDROP
 0001:074E SETCONVERTSTG           SETCONVERTSTG
 0001:1748 SETDOCUMENTBITSTG       SETDOCUMENTBITSTG
 0001:1E26 VALIDATEALLOBJECTS      VALIDATEALLOBJECTS
 0001:0A4C WEP                     WEP
 0001:0098 WRITECLASSSTG           WRITECLASSSTG
 0001:107C WRITECLASSSTM           WRITECLASSSTM
 0001:00BE WRITEFMTUSERTYPESTG     WRITEFMTUSERTYPESTG
 0001:07E6 WRITEOLESTG             WRITEOLESTG
 0001:1C18 WRITESTRINGSTREAM       WRITESTRINGSTREAM
 0001:52A0 XFORMHEIGHTINHIMETRICTOPIXELS  XFORMHEIGHTINHIMETRICTOPIXELS
 0001:524A XFORMHEIGHTINPIXELSTOHIMETRIC  XFORMHEIGHTINPIXELSTOHIMETRIC
 0001:51F4 XFORMWIDTHINHIMETRICTOPIXELS  XFORMWIDTHINHIMETRICTOPIXELS
 0001:519E XFORMWIDTHINPIXELSTOHIMETRIC  XFORMWIDTHINPIXELSTOHIMETRIC
 0001:0B12 _IID_IAdviseSink        _IID_IAdviseSink
 0001:0BF2 _IID_IAdviseSink2       _IID_IAdviseSink2
 0001:0AF2 _IID_IDataAdviseHolder  _IID_IDataAdviseHolder
 0001:0B42 _IID_IDataObject        _IID_IDataObject
 0001:0C52 _IID_IDebug             _IID_IDebug
 0001:0C22 _IID_IDebugStream       _IID_IDebugStream
 0001:0C92 _IID_IDropSource        _IID_IDropSource
 0001:0C72 _IID_IDropTarget        _IID_IDropTarget
 0001:0C82 _IID_IEnumCallback      _IID_IEnumCallback
 0001:0D62 _IID_IEnumFORMATETC     _IID_IEnumFORMATETC
 0001:0CD2 _IID_IEnumGeneric       _IID_IEnumGeneric
 0001:0CB2 _IID_IEnumHolder        _IID_IEnumHolder
 0001:0D92 _IID_IEnumMoniker       _IID_IEnumMoniker
 0001:0D32 _IID_IEnumOLEVERB       _IID_IEnumOLEVERB
 0001:0D02 _IID_IEnumSTATDATA      _IID_IEnumSTATDATA
 0001:0DC2 _IID_IEnumString        _IID_IEnumString
 0001:0E02 _IID_IEnumUnknown       _IID_IEnumUnknown
 0001:0AC2 _IID_IOleAdviseHolder   _IID_IOleAdviseHolder
 0001:0D22 _IID_IOleCache          _IID_IOleCache
 0001:0B62 _IID_IOleCache2         _IID_IOleCache2
 0001:0B32 _IID_IOleCacheControl   _IID_IOleCacheControl
 0001:0E32 _IID_IOleClientSite     _IID_IOleClientSite
 0001:0DB2 _IID_IOleContainer      _IID_IOleContainer
 0001:0E52 _IID_IOleInPlaceActiveObject  _IID_IOleInPlaceActiveObject
 0001:0E72 _IID_IOleInPlaceFrame   _IID_IOleInPlaceFrame
 0001:0A72 _IID_IOleInPlaceObject  _IID_IOleInPlaceObject
 0001:0E12 _IID_IOleInPlaceSite    _IID_IOleInPlaceSite
 0001:0E92 _IID_IOleInPlaceUIWindow  _IID_IOleInPlaceUIWindow
 0001:0D82 _IID_IOleItemContainer  _IID_IOleItemContainer
 0001:0D52 _IID_IOleLink           _IID_IOleLink
 0001:0CF2 _IID_IOleManager        _IID_IOleManager
 0001:0A92 _IID_IOleObject         _IID_IOleObject
 0001:0CC2 _IID_IOlePresObj        _IID_IOlePresObj
 0001:0A52 _IID_IOleWindow         _IID_IOleWindow
 0001:0DE2 _IID_IParseDisplayName  _IID_IParseDisplayName
 0001:0BA2 _IID_IPersist           _IID_IPersist
 0001:0BD2 _IID_IPersistFile       _IID_IPersistFile
 0001:0C12 _IID_IPersistStorage    _IID_IPersistStorage
 0001:0C32 _IID_IPersistStream     _IID_IPersistStream
 0001:0BC2 _IID_IRunnableObject    _IID_IRunnableObject
 0001:0B72 _IID_IViewObject        _IID_IViewObject
 0001:0B82 _IID_IViewObject2       _IID_IViewObject2
 0002:0ABE ___ExportedStub         ___ExportedStub

  Address         Publics by Name

 0003:0000       ??0IStream@@REC@XZ
 0002:00EA       ??2@ZAPEXI@Z
 0002:00D8       ??3@ZAXPEX@Z
 0003:0028       ??_7CMemBytes@@6F@
 0003:005C       ??_7CMemStm@@6F@
 0003:013C       ??_7CMMB@@6F@
 0003:0118       ??_7CMMS@@6F@
 0003:0094       ??_7ILockBytes@@6F@
 0003:00F4       ??_7IMarshal@@6F@
 0003:00BC       ??_7IStream@@6F@
 0003:0050       ??_7IUnknown@@6F@
 0001:3000       ?AddRef@CMemBytes@@VEAKXZ
 0001:23A2       ?AddRef@CMemStm@@VEAKXZ
 0001:3B88       ?AddRef@CMMB@@VEAKXZ
 0001:35F2       ?AddRef@CMMS@@VEAKXZ
 0001:10D4       ?BmDuplicate@@ZAIIPEKPEUtagBITMAP@@@Z
 0001:2B48       ?Clone@CMemStm@@VEAPEXPEPEUIStream@@@Z
 0001:2A3A       ?Commit@CMemStm@@VEAPEXK@Z
 0001:28AA       ?CopyTo@CMemStm@@VEAPEXPEUIStream@@U_ULARGE_INTEGER@@PEU3@2@Z
 0001:3458       ?Create@CMemBytes@@TAPEV1@I@Z
 0001:2BAE       ?Create@CMemStm@@TAPEV1@I@Z
 0001:3F58       ?Create@CMMB@@TAPEV1@PEVCMemBytes@@@Z
 0001:39CA       ?Create@CMMS@@TAPEV1@PEVCMemStm@@@Z
 0001:3F48       ?DisconnectObject@CMMB@@VEAPEXK@Z
 0001:39BA       ?DisconnectObject@CMMS@@VEAPEXK@Z
 0001:44E8       ?FIconFileFromClass@@ZCHAFUGUID@@PEDIPEI@Z
 0001:32E2       ?Flush@CMemBytes@@VEAPEXXZ
 0004:006E       ?gdwOleVersion@@3KE
 0001:4238       ?GetAssociatedExecutable@@ZCHPED0@Z
 0001:3C7C       ?GetMarshalSizeMax@CMMB@@VEAPEXAFUGUID@@PEXK1KPEK@Z
 0001:36E8       ?GetMarshalSizeMax@CMMS@@VEAPEXAFUGUID@@PEXK1KPEK@Z
 0001:3C2C       ?GetUnmarshalClass@CMMB@@VEAPEXAFUGUID@@PEXK1KPEU2@@Z
 0001:3696       ?GetUnmarshalClass@CMMS@@VEAPEXAFUGUID@@PEXK1KPEU2@@Z
 0001:4470       ?HIconAndSourceFromClass@@ZCIAFUGUID@@PEDPEI@Z
 0004:0038       ?hmodOLE2@@3IE
 0001:207E       ?IsMDIAccelerator@@ZAHPEUtagMSG@@PEG@Z
 0001:336E       ?LockRegion@CMemBytes@@VEAPEXU_ULARGE_INTEGER@@0K@Z
 0001:2A5A       ?LockRegion@CMemStm@@VEAPEXU_ULARGE_INTEGER@@0K@Z
 0001:3CD0       ?MarshalInterface@CMMB@@VEAPEXPEUIStream@@AFUGUID@@PEXK2K@Z
 0001:374E       ?MarshalInterface@CMMS@@VEAPEXPEUIStream@@AFUGUID@@PEXK2K@Z
 0001:515A       ?PointerToNthField@@ZCPEDPEDHD@Z
 0001:2F3A       ?QueryInterface@CMemBytes@@VEAPEXAFUGUID@@PEPEX@Z
 0001:22DC       ?QueryInterface@CMemStm@@VEAPEXAFUGUID@@PEPEX@Z
 0001:3AD0       ?QueryInterface@CMMB@@VEAPEXAFUGUID@@PEPEX@Z
 0001:3538       ?QueryInterface@CMMS@@VEAPEXAFUGUID@@PEPEX@Z
 0001:2434       ?Read@CMemStm@@VEAPEXPIXKPEK@Z
 0001:3092       ?ReadAt@CMemBytes@@VEAPEXU_ULARGE_INTEGER@@PIXKPEK@Z
 0001:3022       ?Release@CMemBytes@@VEAKXZ
 0001:23C4       ?Release@CMemStm@@VEAKXZ
 0001:3BAA       ?Release@CMMB@@VEAKXZ
 0001:3614       ?Release@CMMS@@VEAKXZ
 0001:3EEC       ?ReleaseMarshalData@CMMB@@VEAPEXPEUIStream@@@Z
 0001:395E       ?ReleaseMarshalData@CMMS@@VEAPEXPEUIStream@@@Z
 0001:2A4A       ?Revert@CMemStm@@VEAPEXXZ
 0001:26D8       ?Seek@CMemStm@@VEAPEXU_LARGE_INTEGER@@KPEU_ULARGE_INTEGER@@@Z
 0001:32F2       ?SetSize@CMemBytes@@VEAPEXU_ULARGE_INTEGER@@@Z
 0001:2822       ?SetSize@CMemStm@@VEAPEXU_ULARGE_INTEGER@@@Z
 0001:338E       ?Stat@CMemBytes@@VEAPEXPEUtagSTATSTG@@K@Z
 0001:2A7E       ?Stat@CMemStm@@VEAPEXPEUtagSTATSTG@@K@Z
 0001:1AEA       ?StRead@@ZAPEXPEUIStream@@PEXK@Z
 0001:337E       ?UnlockRegion@CMemBytes@@VEAPEXU_ULARGE_INTEGER@@0K@Z
 0001:2A6C       ?UnlockRegion@CMemStm@@VEAPEXU_ULARGE_INTEGER@@0K@Z
 0001:3DC8       ?UnmarshalInterface@CMMB@@VEAPEXPEUIStream@@AFUGUID@@PEPEX@Z
 0001:383A       ?UnmarshalInterface@CMMS@@VEAPEXPEUIStream@@AFUGUID@@PEPEX@Z
 0004:04A8       ?uOleMessage@@3IE
 0001:12B4       ?UtDupGlobal@@ZAIII@Z
 0001:120A       ?UtDupPalette@@ZAII@Z
 0001:20EE       ?wGetOleMenuPtr@@ZAPEUtagOLEMENU@@I@Z
 0001:257C       ?Write@CMemStm@@VEAPEXPJXKPEK@Z
 0001:31CC       ?WriteAt@CMemBytes@@VEAPEXU_ULARGE_INTEGER@@PJXKPEK@Z
 0004:04A6       ?wSignature@@3GE
 0000:0000  Imp  ADDAPPCOMPATFLAG     (COMPOBJ.207)
 0000:0000  Imp  ANSIPREV             (USER.473)
 0001:080C       BINDMONIKER
 0000:0000  Imp  CALLOBJECTINWOW      (COMPOBJ.201)
 0000:0000  Imp  CALLPROC32W          (KERNEL.CALLPROC32W)
 0001:2D06       CLONEMEMSTM
 0000:0000  Imp  CLOSEMETAFILE        (GDI.126)
 0001:4046       CMEMBYTESUNMARSHAL
 0001:3AB8       CMEMSTMUNMARSHAL
 0000:0000  Imp  COBUILDVERSION       (COMPOBJ.1)
 0000:0000  Imp  COGETMALLOC          (COMPOBJ.4)
 0000:0000  Imp  COINITIALIZE         (COMPOBJ.2)
 0000:0000  Imp  COISOLE1CLASS        (COMPOBJ.36)
 0000:0000  Imp  COPYMETAFILE         (GDI.151)
 0000:0000  Imp  COUNINITIALIZE       (COMPOBJ.3)
 0001:09BE       CREATEANTIMONIKER
 0001:08A4       CREATEBINDCTX
 0000:0000  Imp  CREATEBITMAP         (GDI.48)
 0001:0774       CREATEDATAADVISEHOLDER
 0001:079A       CREATEDATACACHE
 0001:0916       CREATEFILEMONIKER
 0000:0000  Imp  CREATEFONT           (GDI.56)
 0001:08CA       CREATEGENERICCOMPOSITE
 0001:212A       CREATEILOCKBYTESONHGLOBAL
 0001:0998       CREATEITEMMONIKER
 0001:2C84       CREATEMEMSTM
 0000:0000  Imp  CREATEMETAFILE       (GDI.125)
 0001:053A       CREATEOLEADVISEHOLDER
 0000:0000  Imp  CREATEPALETTE        (GDI.360)
 0001:09E4       CREATEPOINTERMONIKER
 0001:2D8E       CREATESTREAMONHGLOBAL
 0000:0000  Imp  CREATEWINDOW         (USER.41)
 0001:1E0C       DBGDUMPCLASSNAME
 0001:1DEC       DBGDUMPEXTERNALOBJECT
 0001:1DDE       DBGDUMPOBJECT
 0001:1DFA       DBGISOBJECTVALID
 0001:1D74       DBGLOGCLOSE
 0001:1D62       DBGLOGOPEN
 0001:1DAC       DBGLOGOUTPUTDEBUGSTRING
 0001:1D90       DBGLOGTIMESTAMP
 0001:1D82       DBGLOGWRITE
 0001:1D9E       DBGLOGWRITEBANNER
 0000:0000  Imp  DEFWINDOWPROC        (USER.107)
 0000:0000  Imp  DELETEMETAFILE       (GDI.127)
 0000:0000  Imp  DELETEOBJECT         (GDI.69)
 0000:0000  Imp  DESTROYICON          (USER.457)
 0001:004C       DLLGETCLASSOBJECT
 0001:0390       DODRAGDROP
 0000:0000  Imp  DOS3CALL             (KERNEL.102)
 0000:0000  Imp  DRAWICON             (USER.84)
 0001:1E1A       DUMPALLOBJECTS
 0000:0000  Imp  ESCAPE               (GDI.38)
 0000:0000  Imp  EXTRACTICON          (SHELL.34)
 0000:0000  Imp  EXTTEXTOUT           (GDI.351)
 0000:0000  Imp  FATALAPPEXIT         (KERNEL.137)
 0000:0000  Imp  FATALEXIT            (KERNEL.1)
 0000:0000  Imp  FREELIBRARY32W       (KERNEL.FREELIBRARY32W)
 0000:0000  Imp  GETBITMAPBITS        (GDI.74)
 0000:0000  Imp  GETBITMAPDIMENSIONEX (GDI.468)
 0001:08F0       GETCLASSFILE
 0001:0728       GETCONVERTSTG
 0000:0000  Imp  GETDC                (USER.66)
 0000:0000  Imp  GETDEVICECAPS        (GDI.80)
 0001:170A       GETDOCUMENTBITSTG
 0000:0000  Imp  GETDOSENVIRONMENT    (KERNEL.131)
 0001:2240       GETHGLOBALFROMILOCKBYTES
 0001:2EA4       GETHGLOBALFROMSTREAM
 0000:0000  Imp  GETKEYSTATE          (USER.106)
 0000:0000  Imp  GETMODULEFILENAME    (KERNEL.49)
 0000:0000  Imp  GETOBJECT            (GDI.82)
 0000:0000  Imp  GETPALETTEENTRIES    (GDI.363)
 0000:0000  Imp  GETPROCADDRESS32W    (KERNEL.GETPROCADDRESS32W)
 0001:0A0A       GETRUNNINGOBJECTTABLE
 0000:0000  Imp  GETSTOCKOBJECT       (GDI.87)
 0000:0000  Imp  GETSYSCOLOR          (USER.180)
 0000:0000  Imp  GETSYSTEMMETRICS     (USER.179)
 0000:0000  Imp  GETTEXTEXTENTPOINT   (GDI.471)
 0000:0000  Imp  GETVDMPOINTER32W     (KERNEL.GETVDMPOINTER32W)
 0000:0000  Imp  GETVERSION           (KERNEL.3)
 0000:0000  Imp  GLOBALALLOC          (KERNEL.15)
 0000:0000  Imp  GLOBALFREE           (KERNEL.17)
 0000:0000  Imp  GLOBALHANDLE         (KERNEL.21)
 0000:0000  Imp  GLOBALLOCK           (KERNEL.18)
 0000:0000  Imp  GLOBALREALLOC        (KERNEL.16)
 0000:0000  Imp  GLOBALSIZE           (KERNEL.20)
 0000:0000  Imp  GLOBALUNLOCK         (KERNEL.19)
 0000:0000  Imp  HMEMCPY              (KERNEL.348)
 0000:0000  Imp  INITAPP              (USER.5)
 0000:0000  Imp  INITTASK             (KERNEL.91)
 0001:1F16       ISACCELERATOR
 0000:0000  Imp  ISBADREADPTR         (KERNEL.334)
 0000:0000  Imp  ISBADWRITEPTR        (KERNEL.335)
 0000:0000  Imp  ISVALIDIID           (COMPOBJ.24)
 0000:0000  Imp  ISVALIDINTERFACE     (COMPOBJ.23)
 0001:0A30       LIBMAIN
 0000:0000  Imp  LOADICON             (USER.174)
 0000:0000  Imp  LOADLIBRARYEX32W     (KERNEL.LOADLIBRARYEX32W)
 0000:0000  Imp  LOCKRESOURCE         (KERNEL.62)
 0000:0000  Imp  LOCKSEGMENT          (KERNEL.23)
 0000:0000  Imp  LOOKUPETASK          (COMPOBJ.94)
 0000:0000  Imp  LSTRCAT              (KERNEL.89)
 0000:0000  Imp  LSTRCPY              (KERNEL.88)
 0000:0000  Imp  LSTRCPYN             (KERNEL.353)
 0000:0000  Imp  LSTRLEN              (KERNEL.90)
 0001:1DCC       MAKEDEBUGSTREAM
 0001:0832       MKPARSEDISPLAYNAME
 0001:087E       MONIKERCOMMONPREFIXWITH
 0001:0858       MONIKERRELATIVEPATHTO
 0000:0000  Imp  MULDIV               (GDI.128)
 0001:10C2       OLEBUILDVERSION
 0001:0644       OLECONVERTISTORAGETOOLESTREAM
 0001:0690       OLECONVERTISTORAGETOOLESTREAMEX
 0001:066A       OLECONVERTOLESTREAMTOISTORAGE
 0001:06B6       OLECONVERTOLESTREAMTOISTORAGEEX
 0001:0156       OLECREATE
 0001:0560       OLECREATEDEFAULTHANDLER
 0001:0586       OLECREATEEMBEDDINGHELPER
 0001:017C       OLECREATEFROMDATA
 0001:023A       OLECREATEFROMFILE
 0001:01EE       OLECREATELINK
 0001:01A2       OLECREATELINKFROMDATA
 0001:0214       OLECREATELINKTOFILE
 0001:0000       OLECREATEMENUDESCRIPTOR
 0001:01C8       OLECREATESTATICFROMDATA
 0001:0026       OLEDESTROYMENUDESCRIPTOR
 0001:196C       OLEDOAUTOCONVERT
 0001:04A2       OLEDRAW
 0001:1344       OLEDUPLICATEDATA
 0001:043C       OLEFLUSHCLIPBOARD
 0001:06DC       OLEGETAUTOCONVERT
 0001:1DBA       OLEGETCLASSID
 0001:0416       OLEGETCLIPBOARD
 0001:435E       OLEGETICONOFCLASS
 0001:405E       OLEGETICONOFFILE
 0001:10A2       OLEGETMALLOC
 0001:0EB2       OLEINITIALIZE
 0001:0456       OLEISCURRENTCLIPBOARD
 0001:04EE       OLEISRUNNING
 0001:0260       OLELOAD
 0001:02AC       OLELOADFROMSTREAM
 0001:0514       OLELOCKRUNNING
 0001:4838       OLEMETAFILEPICTFROMICONANDLABEL
 0001:031E       OLENOTEOBJECTVISIBLE
 0001:0130       OLEQUERYCREATEFROMDATA
 0001:010A       OLEQUERYLINKFROMDATA
 0001:05F8       OLEREGENUMFORMATETC
 0001:061E       OLEREGENUMVERBS
 0001:05D2       OLEREGGETMISCSTATUS
 0001:05AC       OLEREGGETUSERTYPE
 0001:04C8       OLERUN
 0001:0286       OLESAVE
 0001:02D2       OLESAVETOSTREAM
 0001:0702       OLESETAUTOCONVERT
 0001:03B6       OLESETCLIPBOARD
 0001:02F8       OLESETCONTAINEDOBJECT
 0001:047C       OLESETMENUDESCRIPTOR
 0001:502C       OLESTDGETAUXUSERTYPE
 0001:4EB8       OLESTDGETUSERTYPEOFCLASS
 0001:4B1E       OLESTDICONLABELTEXTOUT
 0001:1E38       OLETRANSLATEACCELERATOR
 0001:0FFE       OLEUNINITIALIZE
 0000:0000  Imp  OPENFILE             (KERNEL.74)
 0001:1CE4       OPENORCREATESTREAM
 0000:0000  Imp  PROGIDFROMCLSID      (COMPOBJ.62)
 0001:0072       READCLASSSTG
 0001:1056       READCLASSSTM
 0001:00E4       READFMTUSERTYPESTG
 0001:07C0       READOLESTG
 0001:1B3A       READSTRINGSTREAM
 0000:0000  Imp  REGCLOSEKEY          (SHELL.3)
 0000:0000  Imp  REGISTERCLASS        (USER.57)
 0001:0344       REGISTERDRAGDROP
 0000:0000  Imp  REGISTERWINDOWMESSAGE (USER.118)
 0000:0000  Imp  REGOPENKEY           (SHELL.1)
 0000:0000  Imp  REGQUERYVALUE        (SHELL.6)
 0000:0000  Imp  RELEASEDC            (USER.68)
 0001:2D1C       RELEASEMEMSTM
 0001:1784       RELEASESTGMEDIUM
 0001:036A       REVOKEDRAGDROP
 0004:0004       rsrvptrs
 0000:0000  Imp  SELECTOBJECT         (GDI.45)
 0000:0000  Imp  SENDMESSAGE          (USER.111)
 0000:0000  Imp  SETBITMAPBITS        (GDI.106)
 0000:0000  Imp  SETBITMAPDIMENSIONEX (GDI.478)
 0000:0000  Imp  SETBKMODE            (GDI.2)
 0001:074E       SETCONVERTSTG
 0001:1748       SETDOCUMENTBITSTG
 0000:0000  Imp  SETETASK             (COMPOBJ.95)
 0000:0000  Imp  SETRECTEMPTY         (USER.73)
 0000:0000  Imp  SETTEXTCOLOR         (GDI.9)
 0000:0000  Imp  SETWINDOWEXTEX       (GDI.481)
 0000:0000  Imp  SETWINDOWORGEX       (GDI.482)
 0000:0000  Imp  STRINGFROMCLSID      (COMPOBJ.19)
 0001:1E26       VALIDATEALLOBJECTS
 0000:0000  Imp  WAITEVENT            (KERNEL.30)
 0001:0A4C       WEP
 0001:0098       WRITECLASSSTG
 0001:107C       WRITECLASSSTM
 0001:00BE       WRITEFMTUSERTYPESTG
 0001:07E6       WRITEOLESTG
 0001:1C18       WRITESTRINGSTREAM
 0001:52A0       XFORMHEIGHTINHIMETRICTOPIXELS
 0001:524A       XFORMHEIGHTINPIXELSTOHIMETRIC
 0001:51F4       XFORMWIDTHINHIMETRICTOPIXELS
 0001:519E       XFORMWIDTHINPIXELSTOHIMETRIC
 0004:018A       _aseghi
 0004:0188       _aseglo
 0002:00FA       _atoi
 0001:0E62       _CLSID_AntiMoniker
 0001:0DF2       _CLSID_CompositeMoniker
 0001:0DD2       _CLSID_DfMarshal
 0001:0B52       _CLSID_ExcelChart
 0001:0B22       _CLSID_ExcelMacrosheet
 0001:0B92       _CLSID_ExcelWorksheet
 0001:0EA2       _CLSID_FileMoniker
 0001:0E82       _CLSID_ItemMoniker
 0001:0BE2       _CLSID_MSDraw
 0001:0BB2       _CLSID_Package
 0001:0E22       _CLSID_PackagerMoniker
 0001:0AE2       _CLSID_PBrush
 0001:0AB2       _CLSID_Picture_Dib
 0001:0B02       _CLSID_Picture_Metafile
 0001:0E42       _CLSID_PointerMoniker
 0001:0C62       _CLSID_PSBindCtx
 0001:0D42       _CLSID_PSClassObject
 0001:0D72       _CLSID_PSClientSite
 0001:0CA2       _CLSID_PSDragDrop
 0001:0C42       _CLSID_PSEnumerators
 0001:0DA2       _CLSID_PSGenObject
 0001:0D12       _CLSID_PSInPlaceActive
 0001:0CE2       _CLSID_PSInPlaceFrame
 0001:0C02       _CLSID_PSStore
 0001:0A62       _CLSID_StdMemBytes
 0001:0A82       _CLSID_StdMemStm
 0001:0AA2       _CLSID_StdOleLink
 0001:0AD2       _CLSID_WordDocument
 0004:04A6       _edata
 0004:04E2       _end
 0004:02AE       _errno
 0002:0317       _exit
 0000:0000  Imp  _GUID_NULL           (COMPOBJ.37)
 0001:0B12       _IID_IAdviseSink
 0001:0BF2       _IID_IAdviseSink2
 0001:0AF2       _IID_IDataAdviseHolder
 0001:0B42       _IID_IDataObject
 0001:0C52       _IID_IDebug
 0001:0C22       _IID_IDebugStream
 0001:0C92       _IID_IDropSource
 0001:0C72       _IID_IDropTarget
 0001:0C82       _IID_IEnumCallback
 0001:0D62       _IID_IEnumFORMATETC
 0001:0CD2       _IID_IEnumGeneric
 0001:0CB2       _IID_IEnumHolder
 0001:0D92       _IID_IEnumMoniker
 0001:0D32       _IID_IEnumOLEVERB
 0001:0D02       _IID_IEnumSTATDATA
 0001:0DC2       _IID_IEnumString
 0001:0E02       _IID_IEnumUnknown
 0000:0000  Imp  _IID_ILockBytes      (COMPOBJ.48)
 0000:0000  Imp  _IID_IMarshal        (COMPOBJ.41)
 0001:0AC2       _IID_IOleAdviseHolder
 0001:0D22       _IID_IOleCache
 0001:0B62       _IID_IOleCache2
 0001:0B32       _IID_IOleCacheControl
 0001:0E32       _IID_IOleClientSite
 0001:0DB2       _IID_IOleContainer
 0001:0E52       _IID_IOleInPlaceActiveObject
 0001:0E72       _IID_IOleInPlaceFrame
 0001:0A72       _IID_IOleInPlaceObject
 0001:0E12       _IID_IOleInPlaceSite
 0001:0E92       _IID_IOleInPlaceUIWindow
 0001:0D82       _IID_IOleItemContainer
 0001:0D52       _IID_IOleLink
 0001:0CF2       _IID_IOleManager
 0001:0A92       _IID_IOleObject
 0001:0CC2       _IID_IOlePresObj
 0001:0A52       _IID_IOleWindow
 0001:0DE2       _IID_IParseDisplayName
 0001:0BA2       _IID_IPersist
 0001:0BD2       _IID_IPersistFile
 0001:0C12       _IID_IPersistStorage
 0001:0C32       _IID_IPersistStream
 0001:0BC2       _IID_IRunnableObject
 0000:0000  Imp  _IID_IStream         (COMPOBJ.50)
 0000:0000  Imp  _IID_IUnknown        (COMPOBJ.38)
 0001:0B72       _IID_IViewObject
 0001:0B82       _IID_IViewObject2
 0004:017C       _STKHQQ
 0002:00FE       _strcspn
 0000:0000  Imp  _wsprintf            (USER.420)
 0004:0292       __acfinfo
 0000:9876  Abs  __acrtmsg
 0000:9876  Abs  __acrtused
 0000:D6D6  Abs  __aDBdoswp
 0004:0300       __adbgmsg
 0000:D6D6  Abs  __aDBused
 0002:0160       __aFlmul
 0002:0160       __aFulmul
 0000:0000  Imp  __AHINCR             (KERNEL.114)
 0000:0000  Imp  __AHSHIFT            (KERNEL.113)
 0004:02A0       __aintdiv
 0004:031C       __amblksiz
 0002:0684       __amsg_exit
 0002:001A       __astart
 0002:078E       __catox
 0002:0334       __cexit
 0004:02FD       __child
 0002:0234       __cinit
 0002:067A       __cintDIV
 0004:0186       __cmdShow
 0004:02BD       __cpumode
 0002:03B5       __ctermsub
 0004:0190       __ctype
 0004:0190       __ctype_
 0002:0345       __c_exit
 0004:02BE       __doserrno
 0004:04A6       __edata
 0004:04E2       __end
 0004:02F4       __environ
 0002:0325       __exit
 0004:02FF       __exitflag
 0004:02A4       __fac
 0002:06C6       __ffree
 0002:03F2       __FF_MSGBANNER
 0004:030E       __fheap
 0002:0A1B       __findlast
 0002:06E7       __fmalloc
 0002:0192       __fmemcmp
 0004:0320       __fpinit
 0000:9876  Abs  __fptaskdata
 0002:07F0       __fptrap
 0002:015A       __fpurecall
 0002:01EE       __fstrlen
 0002:0898       __GetDGROUP
 0002:0924       __growseg
 0004:0180       __hInstance
 0004:017E       __hPrevInstance
 0002:09B5       __incseg
 0002:0AD2       __initseg
 0002:0B06       __linkseg
 0004:0182       __lpszCmdLine
 0002:086A       __myalloc
 0002:0A3C       __newseg
 0004:02C0       __nfile
 0002:07F6       __NMSG_TEXT
 0002:082D       __NMSG_WRITE
 0002:00D1       __nomain
 0002:015A       __npurecall
 0004:02BE       __oserr
 0004:02C6       __osfile
 0004:02B9       __osmajor
 0004:02B8       __osminor
 0004:02BC       __osmode
 0004:02B8       __osver
 0004:02BA       __osversion
 0004:02F8       __pgmptr
 0004:0308       __pnhFarHeap
 0004:02B4       __psp
 0004:02B2       __pspadr
 0002:015A       __purecall
 0002:07E9       __QWINClose
 0002:07E9       __QWINExit
 0002:07E9       __QWINGetBuffSize
 0002:07E9       __QWINGetFocus
 0002:07E9       __QWINGetSize
 0002:07E9       __QWINInit
 0002:07E9       __QWINIsQWINin
 0002:07E9       __QWINMenuClick
 0002:07E9       __QWINOpen
 0002:07E9       __QWINRead
 0002:07E9       __QWINSetAboutString
 0002:07E9       __QWINSetBuffSize
 0002:07E9       __QWINSetFocus
 0002:07E9       __QWINSetSize
 0002:07E9       __QWINTerm
 0004:030C       __qwinused
 0002:07E9       __QWINWrite
 0002:07E9       __QWINYield
 0002:08A8       __searchseg
 0002:0416       __setargv
 0002:05C0       __setenvp
 0000:0001  Abs  __sizec
 0000:0001  Abs  __sized
 0002:0208       __stubmain
 0004:02B0       __umaskval
 0002:07E9       __wabout
 0002:07E4       __wcexit
 0002:07E4       __wcinit
 0002:07E9       __wclose
 0004:02C2       __wfile
 0002:0010       __wflags
 0002:07E9       __wgetfocus
 0002:07E9       __wgetscreenbuf
 0002:07E9       __wgetsize
 0000:0000  Imp  __WINFLAGS           (KERNEL.178)
 0004:02B7       __winmajor
 0004:02B6       __winminor
 0004:02B6       __winver
 0000:0000  Abs  __wiobused
 0002:07E9       __wmenuclick
 0004:02C4       __wnfile
 0002:07E9       __wopen
 0002:07E9       __wread
 0002:07E9       __wsetfocus
 0002:07E9       __wsetscreenbuf
 0002:07E9       __wsetsize
 0004:02DA       __wsfile
 0002:07E9       __wterm
 0002:07E9       __wwrite
 0004:018E       ___aDBrterr
 0004:018C       ___aDBswpflg
 0004:02EE       ___argc
 0004:02F0       ___argv
 0002:0ABE       ___ExportedStub

  Address         Publics by Value

 0000:0000  Imp  STRINGFROMCLSID      (COMPOBJ.19)
 0000:0000  Imp  ISVALIDIID           (COMPOBJ.24)
 0000:0000  Imp  EXTRACTICON          (SHELL.34)
 0000:0000  Imp  WAITEVENT            (KERNEL.30)
 0000:0000  Imp  RELEASEDC            (USER.68)
 0000:0000  Imp  _IID_IStream         (COMPOBJ.50)
 0000:0000  Imp  FATALAPPEXIT         (KERNEL.137)
 0000:0000  Imp  ANSIPREV             (USER.473)
 0000:0000  Imp  PROGIDFROMCLSID      (COMPOBJ.62)
 0000:0000  Imp  GLOBALFREE           (KERNEL.17)
 0000:0000  Imp  REGISTERWINDOWMESSAGE (USER.118)
 0000:0000  Imp  SETWINDOWORGEX       (GDI.482)
 0000:0000  Imp  _IID_ILockBytes      (COMPOBJ.48)
 0000:0000  Imp  _IID_IUnknown        (COMPOBJ.38)
 0000:0000  Imp  SETBITMAPDIMENSIONEX (GDI.478)
 0000:0000  Imp  SETETASK             (COMPOBJ.95)
 0000:0000  Imp  COUNINITIALIZE       (COMPOBJ.3)
 0000:0000  Imp  GETVDMPOINTER32W     (KERNEL.GETVDMPOINTER32W)
 0000:0000  Imp  GETBITMAPDIMENSIONEX (GDI.468)
 0000:0000  Imp  ISBADREADPTR         (KERNEL.334)
 0000:0000  Imp  LOCKRESOURCE         (KERNEL.62)
 0000:0000  Imp  FATALEXIT            (KERNEL.1)
 0000:0000  Imp  ISBADWRITEPTR        (KERNEL.335)
 0000:0000  Imp  DELETEMETAFILE       (GDI.127)
 0000:0000  Imp  GETSYSTEMMETRICS     (USER.179)
 0000:0000  Imp  DESTROYICON          (USER.457)
 0000:0000  Imp  REGISTERCLASS        (USER.57)
 0000:0000  Imp  DOS3CALL             (KERNEL.102)
 0000:0000  Imp  LOADICON             (USER.174)
 0000:0000  Imp  CREATEFONT           (GDI.56)
 0000:0000  Imp  GETPALETTEENTRIES    (GDI.363)
 0000:0000  Imp  CREATEPALETTE        (GDI.360)
 0000:0000  Imp  HMEMCPY              (KERNEL.348)
 0000:0000  Imp  COGETMALLOC          (COMPOBJ.4)
 0000:0000  Imp  __WINFLAGS           (KERNEL.178)
 0000:0000  Imp  __AHSHIFT            (KERNEL.113)
 0000:0000  Imp  SETRECTEMPTY         (USER.73)
 0000:0000  Imp  SELECTOBJECT         (GDI.45)
 0000:0000  Imp  FREELIBRARY32W       (KERNEL.FREELIBRARY32W)
 0000:0000  Imp  GLOBALUNLOCK         (KERNEL.19)
 0000:0000  Imp  _GUID_NULL           (COMPOBJ.37)
 0000:0000  Imp  LOADLIBRARYEX32W     (KERNEL.LOADLIBRARYEX32W)
 0000:0000  Imp  LSTRLEN              (KERNEL.90)
 0000:0000  Imp  DELETEOBJECT         (GDI.69)
 0000:0000  Imp  SETTEXTCOLOR         (GDI.9)
 0000:0000  Imp  MULDIV               (GDI.128)
 0000:0000  Imp  GETPROCADDRESS32W    (KERNEL.GETPROCADDRESS32W)
 0000:0000  Imp  INITAPP              (USER.5)
 0000:0000  Imp  EXTTEXTOUT           (GDI.351)
 0000:0000  Imp  LOCKSEGMENT          (KERNEL.23)
 0000:0000  Imp  SETBKMODE            (GDI.2)
 0000:0000  Imp  GETSTOCKOBJECT       (GDI.87)
 0000:0000  Imp  __AHINCR             (KERNEL.114)
 0000:0000  Imp  LSTRCPYN             (KERNEL.353)
 0000:0000  Imp  LSTRCAT              (KERNEL.89)
 0000:0000  Imp  OPENFILE             (KERNEL.74)
 0000:0000  Imp  LSTRCPY              (KERNEL.88)
 0000:0000  Imp  SENDMESSAGE          (USER.111)
 0000:0000  Imp  GLOBALALLOC          (KERNEL.15)
 0000:0000  Imp  GLOBALREALLOC        (KERNEL.16)
 0000:0000  Imp  LOOKUPETASK          (COMPOBJ.94)
 0000:0000  Imp  INITTASK             (KERNEL.91)
 0000:0000  Imp  GETVERSION           (KERNEL.3)
 0000:0000  Imp  GETKEYSTATE          (USER.106)
 0000:0000  Imp  ESCAPE               (GDI.38)
 0000:0000  Imp  REGOPENKEY           (SHELL.1)
 0000:0000  Imp  ADDAPPCOMPATFLAG     (COMPOBJ.207)
 0000:0000  Imp  CLOSEMETAFILE        (GDI.126)
 0000:0000  Imp  CALLOBJECTINWOW      (COMPOBJ.201)
 0000:0000  Imp  CALLPROC32W          (KERNEL.CALLPROC32W)
 0000:0000  Imp  COPYMETAFILE         (GDI.151)
 0000:0000  Imp  GETSYSCOLOR          (USER.180)
 0000:0000  Imp  ISVALIDINTERFACE     (COMPOBJ.23)
 0000:0000  Abs  __wiobused
 0000:0000  Imp  DEFWINDOWPROC        (USER.107)
 0000:0000  Imp  COBUILDVERSION       (COMPOBJ.1)
 0000:0000  Imp  COISOLE1CLASS        (COMPOBJ.36)
 0000:0000  Imp  REGCLOSEKEY          (SHELL.3)
 0000:0000  Imp  CREATEBITMAP         (GDI.48)
 0000:0000  Imp  GLOBALHANDLE         (KERNEL.21)
 0000:0000  Imp  REGQUERYVALUE        (SHELL.6)
 0000:0000  Imp  CREATEMETAFILE       (GDI.125)
 0000:0000  Imp  COINITIALIZE         (COMPOBJ.2)
 0000:0000  Imp  GETMODULEFILENAME    (KERNEL.49)
 0000:0000  Imp  GETBITMAPBITS        (GDI.74)
 0000:0000  Imp  SETBITMAPBITS        (GDI.106)
 0000:0000  Imp  DRAWICON             (USER.84)
 0000:0000  Imp  GLOBALLOCK           (KERNEL.18)
 0000:0000  Imp  SETWINDOWEXTEX       (GDI.481)
 0000:0000  Imp  GLOBALSIZE           (KERNEL.20)
 0000:0000  Imp  CREATEWINDOW         (USER.41)
 0000:0000  Imp  GETDOSENVIRONMENT    (KERNEL.131)
 0000:0000  Imp  GETDEVICECAPS        (GDI.80)
 0000:0000  Imp  GETDC                (USER.66)
 0000:0000  Imp  _IID_IMarshal        (COMPOBJ.41)
 0000:0000  Imp  GETOBJECT            (GDI.82)
 0000:0000  Imp  GETTEXTEXTENTPOINT   (GDI.471)
 0000:0000  Imp  _wsprintf            (USER.420)
 0000:0001  Abs  __sized
 0000:0001  Abs  __sizec
 0000:9876  Abs  __acrtmsg
 0000:9876  Abs  __fptaskdata
 0000:9876  Abs  __acrtused
 0000:D6D6  Abs  __aDBdoswp
 0000:D6D6  Abs  __aDBused
 0001:0000       OLECREATEMENUDESCRIPTOR
 0001:0026       OLEDESTROYMENUDESCRIPTOR
 0001:004C       DLLGETCLASSOBJECT
 0001:0072       READCLASSSTG
 0001:0098       WRITECLASSSTG
 0001:00BE       WRITEFMTUSERTYPESTG
 0001:00E4       READFMTUSERTYPESTG
 0001:010A       OLEQUERYLINKFROMDATA
 0001:0130       OLEQUERYCREATEFROMDATA
 0001:0156       OLECREATE
 0001:017C       OLECREATEFROMDATA
 0001:01A2       OLECREATELINKFROMDATA
 0001:01C8       OLECREATESTATICFROMDATA
 0001:01EE       OLECREATELINK
 0001:0214       OLECREATELINKTOFILE
 0001:023A       OLECREATEFROMFILE
 0001:0260       OLELOAD
 0001:0286       OLESAVE
 0001:02AC       OLELOADFROMSTREAM
 0001:02D2       OLESAVETOSTREAM
 0001:02F8       OLESETCONTAINEDOBJECT
 0001:031E       OLENOTEOBJECTVISIBLE
 0001:0344       REGISTERDRAGDROP
 0001:036A       REVOKEDRAGDROP
 0001:0390       DODRAGDROP
 0001:03B6       OLESETCLIPBOARD
 0001:0416       OLEGETCLIPBOARD
 0001:043C       OLEFLUSHCLIPBOARD
 0001:0456       OLEISCURRENTCLIPBOARD
 0001:047C       OLESETMENUDESCRIPTOR
 0001:04A2       OLEDRAW
 0001:04C8       OLERUN
 0001:04EE       OLEISRUNNING
 0001:0514       OLELOCKRUNNING
 0001:053A       CREATEOLEADVISEHOLDER
 0001:0560       OLECREATEDEFAULTHANDLER
 0001:0586       OLECREATEEMBEDDINGHELPER
 0001:05AC       OLEREGGETUSERTYPE
 0001:05D2       OLEREGGETMISCSTATUS
 0001:05F8       OLEREGENUMFORMATETC
 0001:061E       OLEREGENUMVERBS
 0001:0644       OLECONVERTISTORAGETOOLESTREAM
 0001:066A       OLECONVERTOLESTREAMTOISTORAGE
 0001:0690       OLECONVERTISTORAGETOOLESTREAMEX
 0001:06B6       OLECONVERTOLESTREAMTOISTORAGEEX
 0001:06DC       OLEGETAUTOCONVERT
 0001:0702       OLESETAUTOCONVERT
 0001:0728       GETCONVERTSTG
 0001:074E       SETCONVERTSTG
 0001:0774       CREATEDATAADVISEHOLDER
 0001:079A       CREATEDATACACHE
 0001:07C0       READOLESTG
 0001:07E6       WRITEOLESTG
 0001:080C       BINDMONIKER
 0001:0832       MKPARSEDISPLAYNAME
 0001:0858       MONIKERRELATIVEPATHTO
 0001:087E       MONIKERCOMMONPREFIXWITH
 0001:08A4       CREATEBINDCTX
 0001:08CA       CREATEGENERICCOMPOSITE
 0001:08F0       GETCLASSFILE
 0001:0916       CREATEFILEMONIKER
 0001:0998       CREATEITEMMONIKER
 0001:09BE       CREATEANTIMONIKER
 0001:09E4       CREATEPOINTERMONIKER
 0001:0A0A       GETRUNNINGOBJECTTABLE
 0001:0A30       LIBMAIN
 0001:0A4C       WEP
 0001:0A52       _IID_IOleWindow
 0001:0A62       _CLSID_StdMemBytes
 0001:0A72       _IID_IOleInPlaceObject
 0001:0A82       _CLSID_StdMemStm
 0001:0A92       _IID_IOleObject
 0001:0AA2       _CLSID_StdOleLink
 0001:0AB2       _CLSID_Picture_Dib
 0001:0AC2       _IID_IOleAdviseHolder
 0001:0AD2       _CLSID_WordDocument
 0001:0AE2       _CLSID_PBrush
 0001:0AF2       _IID_IDataAdviseHolder
 0001:0B02       _CLSID_Picture_Metafile
 0001:0B12       _IID_IAdviseSink
 0001:0B22       _CLSID_ExcelMacrosheet
 0001:0B32       _IID_IOleCacheControl
 0001:0B42       _IID_IDataObject
 0001:0B52       _CLSID_ExcelChart
 0001:0B62       _IID_IOleCache2
 0001:0B72       _IID_IViewObject
 0001:0B82       _IID_IViewObject2
 0001:0B92       _CLSID_ExcelWorksheet
 0001:0BA2       _IID_IPersist
 0001:0BB2       _CLSID_Package
 0001:0BC2       _IID_IRunnableObject
 0001:0BD2       _IID_IPersistFile
 0001:0BE2       _CLSID_MSDraw
 0001:0BF2       _IID_IAdviseSink2
 0001:0C02       _CLSID_PSStore
 0001:0C12       _IID_IPersistStorage
 0001:0C22       _IID_IDebugStream
 0001:0C32       _IID_IPersistStream
 0001:0C42       _CLSID_PSEnumerators
 0001:0C52       _IID_IDebug
 0001:0C62       _CLSID_PSBindCtx
 0001:0C72       _IID_IDropTarget
 0001:0C82       _IID_IEnumCallback
 0001:0C92       _IID_IDropSource
 0001:0CA2       _CLSID_PSDragDrop
 0001:0CB2       _IID_IEnumHolder
 0001:0CC2       _IID_IOlePresObj
 0001:0CD2       _IID_IEnumGeneric
 0001:0CE2       _CLSID_PSInPlaceFrame
 0001:0CF2       _IID_IOleManager
 0001:0D02       _IID_IEnumSTATDATA
 0001:0D12       _CLSID_PSInPlaceActive
 0001:0D22       _IID_IOleCache
 0001:0D32       _IID_IEnumOLEVERB
 0001:0D42       _CLSID_PSClassObject
 0001:0D52       _IID_IOleLink
 0001:0D62       _IID_IEnumFORMATETC
 0001:0D72       _CLSID_PSClientSite
 0001:0D82       _IID_IOleItemContainer
 0001:0D92       _IID_IEnumMoniker
 0001:0DA2       _CLSID_PSGenObject
 0001:0DB2       _IID_IOleContainer
 0001:0DC2       _IID_IEnumString
 0001:0DD2       _CLSID_DfMarshal
 0001:0DE2       _IID_IParseDisplayName
 0001:0DF2       _CLSID_CompositeMoniker
 0001:0E02       _IID_IEnumUnknown
 0001:0E12       _IID_IOleInPlaceSite
 0001:0E22       _CLSID_PackagerMoniker
 0001:0E32       _IID_IOleClientSite
 0001:0E42       _CLSID_PointerMoniker
 0001:0E52       _IID_IOleInPlaceActiveObject
 0001:0E62       _CLSID_AntiMoniker
 0001:0E72       _IID_IOleInPlaceFrame
 0001:0E82       _CLSID_ItemMoniker
 0001:0E92       _IID_IOleInPlaceUIWindow
 0001:0EA2       _CLSID_FileMoniker
 0001:0EB2       OLEINITIALIZE
 0001:0FFE       OLEUNINITIALIZE
 0001:1056       READCLASSSTM
 0001:107C       WRITECLASSSTM
 0001:10A2       OLEGETMALLOC
 0001:10C2       OLEBUILDVERSION
 0001:10D4       ?BmDuplicate@@ZAIIPEKPEUtagBITMAP@@@Z
 0001:120A       ?UtDupPalette@@ZAII@Z
 0001:12B4       ?UtDupGlobal@@ZAIII@Z
 0001:1344       OLEDUPLICATEDATA
 0001:170A       GETDOCUMENTBITSTG
 0001:1748       SETDOCUMENTBITSTG
 0001:1784       RELEASESTGMEDIUM
 0001:196C       OLEDOAUTOCONVERT
 0001:1AEA       ?StRead@@ZAPEXPEUIStream@@PEXK@Z
 0001:1B3A       READSTRINGSTREAM
 0001:1C18       WRITESTRINGSTREAM
 0001:1CE4       OPENORCREATESTREAM
 0001:1D62       DBGLOGOPEN
 0001:1D74       DBGLOGCLOSE
 0001:1D82       DBGLOGWRITE
 0001:1D90       DBGLOGTIMESTAMP
 0001:1D9E       DBGLOGWRITEBANNER
 0001:1DAC       DBGLOGOUTPUTDEBUGSTRING
 0001:1DBA       OLEGETCLASSID
 0001:1DCC       MAKEDEBUGSTREAM
 0001:1DDE       DBGDUMPOBJECT
 0001:1DEC       DBGDUMPEXTERNALOBJECT
 0001:1DFA       DBGISOBJECTVALID
 0001:1E0C       DBGDUMPCLASSNAME
 0001:1E1A       DUMPALLOBJECTS
 0001:1E26       VALIDATEALLOBJECTS
 0001:1E38       OLETRANSLATEACCELERATOR
 0001:1F16       ISACCELERATOR
 0001:207E       ?IsMDIAccelerator@@ZAHPEUtagMSG@@PEG@Z
 0001:20EE       ?wGetOleMenuPtr@@ZAPEUtagOLEMENU@@I@Z
 0001:212A       CREATEILOCKBYTESONHGLOBAL
 0001:2240       GETHGLOBALFROMILOCKBYTES
 0001:22DC       ?QueryInterface@CMemStm@@VEAPEXAFUGUID@@PEPEX@Z
 0001:23A2       ?AddRef@CMemStm@@VEAKXZ
 0001:23C4       ?Release@CMemStm@@VEAKXZ
 0001:2434       ?Read@CMemStm@@VEAPEXPIXKPEK@Z
 0001:257C       ?Write@CMemStm@@VEAPEXPJXKPEK@Z
 0001:26D8       ?Seek@CMemStm@@VEAPEXU_LARGE_INTEGER@@KPEU_ULARGE_INTEGER@@@Z
 0001:2822       ?SetSize@CMemStm@@VEAPEXU_ULARGE_INTEGER@@@Z
 0001:28AA       ?CopyTo@CMemStm@@VEAPEXPEUIStream@@U_ULARGE_INTEGER@@PEU3@2@Z
 0001:2A3A       ?Commit@CMemStm@@VEAPEXK@Z
 0001:2A4A       ?Revert@CMemStm@@VEAPEXXZ
 0001:2A5A       ?LockRegion@CMemStm@@VEAPEXU_ULARGE_INTEGER@@0K@Z
 0001:2A6C       ?UnlockRegion@CMemStm@@VEAPEXU_ULARGE_INTEGER@@0K@Z
 0001:2A7E       ?Stat@CMemStm@@VEAPEXPEUtagSTATSTG@@K@Z
 0001:2B48       ?Clone@CMemStm@@VEAPEXPEPEUIStream@@@Z
 0001:2BAE       ?Create@CMemStm@@TAPEV1@I@Z
 0001:2C84       CREATEMEMSTM
 0001:2D06       CLONEMEMSTM
 0001:2D1C       RELEASEMEMSTM
 0001:2D8E       CREATESTREAMONHGLOBAL
 0001:2EA4       GETHGLOBALFROMSTREAM
 0001:2F3A       ?QueryInterface@CMemBytes@@VEAPEXAFUGUID@@PEPEX@Z
 0001:3000       ?AddRef@CMemBytes@@VEAKXZ
 0001:3022       ?Release@CMemBytes@@VEAKXZ
 0001:3092       ?ReadAt@CMemBytes@@VEAPEXU_ULARGE_INTEGER@@PIXKPEK@Z
 0001:31CC       ?WriteAt@CMemBytes@@VEAPEXU_ULARGE_INTEGER@@PJXKPEK@Z
 0001:32E2       ?Flush@CMemBytes@@VEAPEXXZ
 0001:32F2       ?SetSize@CMemBytes@@VEAPEXU_ULARGE_INTEGER@@@Z
 0001:336E       ?LockRegion@CMemBytes@@VEAPEXU_ULARGE_INTEGER@@0K@Z
 0001:337E       ?UnlockRegion@CMemBytes@@VEAPEXU_ULARGE_INTEGER@@0K@Z
 0001:338E       ?Stat@CMemBytes@@VEAPEXPEUtagSTATSTG@@K@Z
 0001:3458       ?Create@CMemBytes@@TAPEV1@I@Z
 0001:3538       ?QueryInterface@CMMS@@VEAPEXAFUGUID@@PEPEX@Z
 0001:35F2       ?AddRef@CMMS@@VEAKXZ
 0001:3614       ?Release@CMMS@@VEAKXZ
 0001:3696       ?GetUnmarshalClass@CMMS@@VEAPEXAFUGUID@@PEXK1KPEU2@@Z
 0001:36E8       ?GetMarshalSizeMax@CMMS@@VEAPEXAFUGUID@@PEXK1KPEK@Z
 0001:374E       ?MarshalInterface@CMMS@@VEAPEXPEUIStream@@AFUGUID@@PEXK2K@Z
 0001:383A       ?UnmarshalInterface@CMMS@@VEAPEXPEUIStream@@AFUGUID@@PEPEX@Z
 0001:395E       ?ReleaseMarshalData@CMMS@@VEAPEXPEUIStream@@@Z
 0001:39BA       ?DisconnectObject@CMMS@@VEAPEXK@Z
 0001:39CA       ?Create@CMMS@@TAPEV1@PEVCMemStm@@@Z
 0001:3AB8       CMEMSTMUNMARSHAL
 0001:3AD0       ?QueryInterface@CMMB@@VEAPEXAFUGUID@@PEPEX@Z
 0001:3B88       ?AddRef@CMMB@@VEAKXZ
 0001:3BAA       ?Release@CMMB@@VEAKXZ
 0001:3C2C       ?GetUnmarshalClass@CMMB@@VEAPEXAFUGUID@@PEXK1KPEU2@@Z
 0001:3C7C       ?GetMarshalSizeMax@CMMB@@VEAPEXAFUGUID@@PEXK1KPEK@Z
 0001:3CD0       ?MarshalInterface@CMMB@@VEAPEXPEUIStream@@AFUGUID@@PEXK2K@Z
 0001:3DC8       ?UnmarshalInterface@CMMB@@VEAPEXPEUIStream@@AFUGUID@@PEPEX@Z
 0001:3EEC       ?ReleaseMarshalData@CMMB@@VEAPEXPEUIStream@@@Z
 0001:3F48       ?DisconnectObject@CMMB@@VEAPEXK@Z
 0001:3F58       ?Create@CMMB@@TAPEV1@PEVCMemBytes@@@Z
 0001:4046       CMEMBYTESUNMARSHAL
 0001:405E       OLEGETICONOFFILE
 0001:4238       ?GetAssociatedExecutable@@ZCHPED0@Z
 0001:435E       OLEGETICONOFCLASS
 0001:4470       ?HIconAndSourceFromClass@@ZCIAFUGUID@@PEDPEI@Z
 0001:44E8       ?FIconFileFromClass@@ZCHAFUGUID@@PEDIPEI@Z
 0001:4838       OLEMETAFILEPICTFROMICONANDLABEL
 0001:4B1E       OLESTDICONLABELTEXTOUT
 0001:4EB8       OLESTDGETUSERTYPEOFCLASS
 0001:502C       OLESTDGETAUXUSERTYPE
 0001:515A       ?PointerToNthField@@ZCPEDPEDHD@Z
 0001:519E       XFORMWIDTHINPIXELSTOHIMETRIC
 0001:51F4       XFORMWIDTHINHIMETRICTOPIXELS
 0001:524A       XFORMHEIGHTINPIXELSTOHIMETRIC
 0001:52A0       XFORMHEIGHTINHIMETRICTOPIXELS
 0002:0010       __wflags
 0002:001A       __astart
 0002:00D1       __nomain
 0002:00D8       ??3@ZAXPEX@Z
 0002:00EA       ??2@ZAPEXI@Z
 0002:00FA       _atoi
 0002:00FE       _strcspn
 0002:015A       __npurecall
 0002:015A       __fpurecall
 0002:015A       __purecall
 0002:0160       __aFulmul
 0002:0160       __aFlmul
 0002:0192       __fmemcmp
 0002:01EE       __fstrlen
 0002:0208       __stubmain
 0002:0234       __cinit
 0002:0317       _exit
 0002:0325       __exit
 0002:0334       __cexit
 0002:0345       __c_exit
 0002:03B5       __ctermsub
 0002:03F2       __FF_MSGBANNER
 0002:0416       __setargv
 0002:05C0       __setenvp
 0002:067A       __cintDIV
 0002:0684       __amsg_exit
 0002:06C6       __ffree
 0002:06E7       __fmalloc
 0002:078E       __catox
 0002:07E4       __wcinit
 0002:07E4       __wcexit
 0002:07E9       __QWINSetBuffSize
 0002:07E9       __QWINExit
 0002:07E9       __QWINRead
 0002:07E9       __wterm
 0002:07E9       __wmenuclick
 0002:07E9       __QWINGetFocus
 0002:07E9       __wgetfocus
 0002:07E9       __wread
 0002:07E9       __QWINGetSize
 0002:07E9       __wclose
 0002:07E9       __QWINWrite
 0002:07E9       __QWINSetSize
 0002:07E9       __QWINClose
 0002:07E9       __QWINOpen
 0002:07E9       __QWINSetAboutString
 0002:07E9       __wwrite
 0002:07E9       __QWINSetFocus
 0002:07E9       __QWINYield
 0002:07E9       __wopen
 0002:07E9       __wsetsize
 0002:07E9       __wgetsize
 0002:07E9       __QWINMenuClick
 0002:07E9       __QWINIsQWINin
 0002:07E9       __QWINInit
 0002:07E9       __wgetscreenbuf
 0002:07E9       __wsetscreenbuf
 0002:07E9       __QWINGetBuffSize
 0002:07E9       __QWINTerm
 0002:07E9       __wsetfocus
 0002:07E9       __wabout
 0002:07F0       __fptrap
 0002:07F6       __NMSG_TEXT
 0002:082D       __NMSG_WRITE
 0002:086A       __myalloc
 0002:0898       __GetDGROUP
 0002:08A8       __searchseg
 0002:0924       __growseg
 0002:09B5       __incseg
 0002:0A1B       __findlast
 0002:0A3C       __newseg
 0002:0ABE       ___ExportedStub
 0002:0AD2       __initseg
 0002:0B06       __linkseg
 0003:0000       ??0IStream@@REC@XZ
 0003:0028       ??_7CMemBytes@@6F@
 0003:0050       ??_7IUnknown@@6F@
 0003:005C       ??_7CMemStm@@6F@
 0003:0094       ??_7ILockBytes@@6F@
 0003:00BC       ??_7IStream@@6F@
 0003:00F4       ??_7IMarshal@@6F@
 0003:0118       ??_7CMMS@@6F@
 0003:013C       ??_7CMMB@@6F@
 0004:0004       rsrvptrs
 0004:0038       ?hmodOLE2@@3IE
 0004:006E       ?gdwOleVersion@@3KE
 0004:017C       _STKHQQ
 0004:017E       __hPrevInstance
 0004:0180       __hInstance
 0004:0182       __lpszCmdLine
 0004:0186       __cmdShow
 0004:0188       _aseglo
 0004:018A       _aseghi
 0004:018C       ___aDBswpflg
 0004:018E       ___aDBrterr
 0004:0190       __ctype
 0004:0190       __ctype_
 0004:0292       __acfinfo
 0004:02A0       __aintdiv
 0004:02A4       __fac
 0004:02AE       _errno
 0004:02B0       __umaskval
 0004:02B2       __pspadr
 0004:02B4       __psp
 0004:02B6       __winminor
 0004:02B6       __winver
 0004:02B7       __winmajor
 0004:02B8       __osver
 0004:02B8       __osminor
 0004:02B9       __osmajor
 0004:02BA       __osversion
 0004:02BC       __osmode
 0004:02BD       __cpumode
 0004:02BE       __oserr
 0004:02BE       __doserrno
 0004:02C0       __nfile
 0004:02C2       __wfile
 0004:02C4       __wnfile
 0004:02C6       __osfile
 0004:02DA       __wsfile
 0004:02EE       ___argc
 0004:02F0       ___argv
 0004:02F4       __environ
 0004:02F8       __pgmptr
 0004:02FD       __child
 0004:02FF       __exitflag
 0004:0300       __adbgmsg
 0004:0308       __pnhFarHeap
 0004:030C       __qwinused
 0004:030E       __fheap
 0004:031C       __amblksiz
 0004:0320       __fpinit
 0004:04A6       ?wSignature@@3GE
 0004:04A6       __edata
 0004:04A6       _edata
 0004:04A8       ?uOleMessage@@3IE
 0004:04E2       _end
 0004:04E2       __end

Program entry point at 0002:001a
